:020000040000FA
:020000000528D1
:08000800912A83129F01831667
:1000100006309F0008308500E030860087018101AE
:100020000C1483121F30900040308B00B001A401EB
:10003000A501A601A701A0018E018F010515851458
:10004000051486018701B7218B17A01D3128861F53
:100050003828B018D628061F4428A801861E642810
:10006000D628B018C22803302005031DAD28D62895
:100070008A22861BD6288519AD28301C3014B0186A
:100080003015861F4128D6288A22061BD628EF2045
:10009000F620851D5128A70A0C3027020319A70155
:1000A0005728A7032709031D57280B30A700201541
:1000B0008B132708B80003218B1720118A22061BF7
:1000C000D6286922692244288A22861AD628EF2057
:1000D0008E018F01A401F620851D86280530280297
:1000E00003187E28A50A0A302502031D9E28A501B3
:1000F000A60A063026020319A6019E280530A50788
:100100000A302502031C9E28A50078280530280205
:1001100003189728A5032509031D9E280930A5006B
:10012000A6032609031D9E280530A6009E2805303B
:10013000A50203189E280A30A507902820158B13C6
:100140002508B6002608B7000A218B1720118A223D
:10015000861AD628A80A69226428EF20F620A0185B
:10016000B3287522F6206922692269228B13270899
:10017000B80003212508B6002608B7000A21482147
:100180008B17D628EF208B13A01FCA283508B8007C
:100190000321D528A01ED2283308B6003408B700A2
:1001A0000A21D528201ED52829218B170514A00146
:1001B000AD080319E028AD03031DE028860187017F
:1001C0008B156300A01DEB280608E039E03A031DFB
:1001D000EB28A011E028071582220711252880307E
:1001E0008700860105100430AD0008006030A300D0
:1001F00087166422642264228712642264226422A5
:10020000A30BF82808000130A9005730AA003808CD
:10021000302108003608031D19293708031D12294B
:10022000502128290130A9007B30AA003703302152
:1002300028293708031922290130A9008A30AA0089
:10024000370330210130A9009930AA00360330214C
:1002500008000130A9008A30AA00320330210800CA
:10026000AB00AB072B07AA070318A90A3930840093
:100270000330AC0044218000840AAA0A0319A90AA9
:10028000AC0B3A29D621080029088A002A088200E6
:100290000230B900DF30BA007030BB00D621080050
:1002A000201D56296922692269226922080000342A
:1002B0000034003400341134D03400341F34F034AE
:1002C00000342934703400343734F034003442348C
:1002D000D03400344D34103400345B34A034003456
:1002E0006A34D03400347A34603400348334403497
:1002F00000348F3400340034A53410340034B53465
:10030000A0340034C93440340034E234D0340234F0
:100310000034003402341134B03402341834F03470
:10032000023425347034023434349034023444348A
:10033000203402344F34903402346034D0340234E8
:100340006D3420340234813490340234903480345B
:100350000234A03450340234B33450340234C13443
:1003600030340234D13400340234DF347034861B2C
:10037000D529861FB929EF206922F6207522F6209B
:1003800069220130A9005730AA00752203013021EB
:10039000B7302A02031DC52901302902031DC529D2
:1003A00069226922F6207522F62008004B221022CD
:1003B0005422A0303904BE001E2254223A08BE0046
:1003C0001E2254223B08BE001E2254221022542218
:1003D000A1303904BE001E2254223C1529223D09B9
:1003E00003190B2AE0302E0587001F302E058600EA
:1003F000AF013D080310AE0703182F14AE0C2F18E1
:10040000AE178522E0302E0587001F302E058600AE
:100410003D08AE00ED293C11292254221822080083
:10042000851454224F220511542285104B220800B6
:100430004F220511851454224B2208000830BF00BA
:100440003C14BE1F3C103822BE0DBF0B202A422296
:100450000800BD010830BF000310BD0D4222BC18CA
:100460003D14BF0B2D2A3C143C193C1038220800C7
:1004700085103C183D2A4F22051185145422851001
:100480004B22080085104B22BC1485145422051DF4
:10049000BC1085100800831605158312080083160A
:1004A0000511831205150800552A562A572A582A7D
:1004B000592A5A2A5B2A5C2A5D2A5E2A5F2A602A08
:1004C000612A622A632A0800A630A100A10B662ACD
:1004D0000800F830A20064226422A20B6B2AF830D4
:1004E000A20064226422A20B712AF830A2006422C6
:1004F0006422A20B772AF830A20064226422A20BA5
:100500007D2A08003030A2007D2A1730A100A10BFF
:10051000872A08006330A20064226422A20B8C2A7E
:100520000800F0000308F1000C189A2A0B108B1138
:10053000A015F42A0C10301CD72A00308E00803011
:100540008F00B018A92AB014B101B301B401B501EC
:10055000D72AB10A3108AB00B2010530AB02031C47
:10056000D02AB20AAB08031DAD2A2016063032028B
:10057000031DD02AB101A016B30A0A303302031DAD
:10058000D02AB3012017B40A06303402031DD02A42
:10059000B401A017B50A0C303502031DD02AB501ED
:1005A0003118F42A301DD72A8E018F01B001A40A18
:1005B0000F302402031DF42AA401A50A0A302502E3
:1005C000031DF42AA501A60A033026020319A0146C
:1005D00006302602031DF42AA601A70A20140C30B7
:1005E0002702031DF42AA70171088300F00E700E84
:0205F000090000
:02400E00323F3F
:00000001FF
